:100000006F00A05400000000B4000000B600000023
:1000100000000000000000000000000000000000E0
:1000200000000000000000000000000000000000D0
:1000300018050000000000001A0500000000000084
:100040001C0500001E050000200500002205000020
:100050002405000026050000280500002A050000F0
:100060002C0500002E0500003005000032050000C0
:100070003405000036050000380500003A05000090
:100080003C0500003E050000400500004205000060
:10009000440500004605000048050000000000007F
:1000A000511126C022C206C4828282441244A24058
:1000B0003101828001A001A0EFF29FFE7111AE8498
:1000C000137405FC552B81473387F4000C4333052B
:1000D000F4003EC0F1238247130700049107E39523
:1000E000E7FE2285CD2B1101C9B7371701409306D2
:1000F0000004232AD74083270740B70610F0FD16D7
:10010000F58FB706A008D58F2320F740B7470140E9
:100110002398078031472396E780239A07801307A7
:10012000000D2394E78003D7C7808966558F2396F7
:10013000E7808280EFF2DFF6370700209307C700E1
:1001400080339C23930610086381D70C63E8F60084
:10015000930600086389D704054581BF9304C7004F
:10016000130720086387E70C13073008E396E7FEC0
:100170002384018C05472382E184B70700083707F1
:1001800000202320F700370700202322F700B7279D
:100190000240984BA1660945558F98CB984B136741
:1001A000070898CB5DBFB704002083D784001307EE
:1001B000C7008146938484001386818493F5F60FEB
:1001C000050763E88504A297C207C1839EA01307B1
:1001D000F0030145E373F7F837040020032504001A
:1001E00093858184D13D9A208147130707FC4207FC
:1001F00041839AA0130404009386818463E2E7029A
:100200001C40938707041CC019A08129312901458E
:10021000A9B72833B385D700B29588A1850679BFE1
:100220003386F60083450604850793F7F70F0CA283
:10023000F1B71387818C1C2385EF854614A33707FC
:1002400000200356870093060004918E1385818455
:10025000FD5263CFD702B707002003A5070093859F
:100260008184993DB7070020138387002310030082
:10027000B706002083A746002687014693864600DE
:100280009375F60F63EF85000145A2979CC2F1B507
:100290003307F500329785072300570093F7F70FD0
:1002A0004DBFB385C70048238C2105060507E30928
:1002B000B5FC0545D9BFEFF2BFDE37440140AA8443
:1002C000930704803E85930500044D21B747014004
:1002D0009387078065D9A685130504804121F1B372
:1002E000EFF21FDC374401409304048093050002C1
:1002F0002685AD2965DD13050480AD211375F50F45
:100300006DB3EFF2FFD9E93F93077005631BF50862
:10031000C13F9307B00A6316F508D937B707002025
:100320009384C70088A02A84653F2A9488B04D3FF3
:100330001374F40FA8A022951374F50F5537982065
:100340002A94B7070020A8B01377D70F93060008A8
:100350001374F40F9387C7006315D702814439A83B
:100360004137B70700209387C700338797002A9447
:10037000850448A31374F40F93F4F40F9833E3E166
:10038000E4FEB93F631F8500753389472A84630AF9
:10039000F50001450D37854705456303F400014528
:1003A000193F21B3EFF2DFCF371702405C53B70696
:1003B00000010145D58F5CD3892EB707EFBE37E723
:1003C00000E0938707083CC7CDB1EFF27FCDC1476E
:1003D000371702401CCF371701405CCB1C43B706D0
:1003E000080093F7F70FD58F1CC3B73601409387EA
:1003F00006C0DA334207418301EB37170140144747
:10040000C18A89E6453701A00100D5B79566371640
:1004100002409386568314CE1146232AC780854511
:100420002328B740832607807D761306F60FF18ECA
:100430000566130606A0D18E2320D78083260740A9
:10044000716513050520C19A93E626002320D74045
:1004500013077002DAB77D579AB7CEAB13070004C3
:100460009AB3794798DF19679AAF61772392E704C7
:10047000130710289AA337440140853913040480D8
:10048000930500022285DD2465FDA53DD5BFEFF271
:100490003FC1371402401C403707FFF8414593E73E
:1004A00017001CC05C40F98F5CC01C403707F7FE8A
:1004B0007D17F98F1CC01C403707FCFF7D17F98F93
:1004C0001CC05C4041777D17F98F5CC0B7079F0067
:1004D0001CC4A52C1C4C93E707021CCCB717014089
:1004E00003A70740938607401377F7F023A0E74060
:1004F00003A707401367070823A0E74089479CCA62
:10050000B72702409843719B98C3984398C35C40B7
:100510005CC061BE01A001A001A001A001A001A0DA
:1005200001A001A001A001A001A001A001A001A0C3
:1005300001A001A001A001A001A001A001A001A0B3
:1005400001A001A001A001A001A0970100209381BA
:10055000E12B138181FF1305807797050020938598
:1005600065AA17060020130666AA63FAC50083224F
:10057000050023A0550011059105E3EAC5FE170506
:1005800000201305A5A89385C18C6377B5002320AF
:1005900005001105E36DB5FE93020008739002306B
:1005A0008D4273904280970200009382A2A593E24D
:1005B000320073905230EFF09FED9702000093826B
:1005C00002E17390123473002030B7076745372774
:1005D0000240938737125CC3B797EFCD9387B79AE2
:1005E0005CC38280372702401C4B93E707081CCB73
:1005F0008280372702405C470545858B91E7484755
:100600004189133515000D058280EFF27FA92A84F8
:10061000CD3785476318F50019E0154529A0D13F6E
:100620007D14C5BF7DD851B4EFF29FA737050B00ED
:10063000E93F91476312F502372402401C48370511
:100640000B0093E747001CC81C4893E707041CC82D
:100650006D3F1C48ED9B1CC889BCB7066745B72792
:100660000240938636123797EFCDD4C31307B79A5B
:10067000D8C3D4D3D8D38280B7270240984BC16661
:10068000558F98CB984BB7060800558F98CBD84715
:10069000058B75FF984BC176FD16758F98CB8280C0
:1006A000B70700F8AA97116763F6E702B727024079
:1006B000984BC166558F98CB0CC1984BB706040078
:1006C000558F98CBD847058B75FF984BC176FD1693
:1006D000758F98CB8280B70700F8AA97116763F5EA
:1006E000E702B7270240984BC166558F98CBC8CB1D
:1006F000984B1367070498CBD847058B75FF984B29
:10070000C176FD16758F98CB8280EFF27F997111BB
:100710002AC0653DB7066745B72702409386361263
:1007200094D7B796EFCD9386B69A94D7D44771767F
:100730007D160245F18ED4C711676315E500D847D1
:10074000498FD8C7453511018DB2371702401C4378
:100750000E0593F777F05D8D08C3828093F5F51F42
:100760004EA182804A211375F51F82800A216D8D6A
:080770003335A0008280000077
:08077800000000080000000869
:00000001FF
